 management_ext

 Timestamp is ffffffff (Sun Feb  7 06:28:15 2106)

 Preferred load address is 10000000

 Start         Length     Name                   Class
 0001:00000000 000027c0H .text$mn                CODE
 0002:00000000 00000100H .idata$5                DATA
 0002:00000100 00000004H .00cfg                  DATA
 0002:00000104 00000004H .CRT$XCA                DATA
 0002:00000108 00000004H .CRT$XCZ                DATA
 0002:0000010c 00000004H .CRT$XIA                DATA
 0002:00000110 00000004H .CRT$XIZ                DATA
 0002:00000114 00000004H .CRT$XPA                DATA
 0002:00000118 00000004H .CRT$XPZ                DATA
 0002:0000011c 00000004H .CRT$XTA                DATA
 0002:00000120 00000010H .CRT$XTZ                DATA
 0002:00000124 00000000H .gfids$y                DATA
 0002:00000130 000007d0H .rdata                  DATA
 0002:00000900 00000004H .rdata$sxdata           DATA
 0002:00000904 0000028cH .rdata$zzzdbg           DATA
 0002:00000b90 00000004H .rtc$IAA                DATA
 0002:00000b94 00000004H .rtc$IZZ                DATA
 0002:00000b98 00000004H .rtc$TAA                DATA
 0002:00000b9c 00000004H .rtc$TZZ                DATA
 0002:00000ba0 00000080H .xdata$x                DATA
 0002:00000c20 00000888H .edata                  DATA
 0002:000014a8 000000dcH .idata$2                DATA
 0002:00001584 00000014H .idata$3                DATA
 0002:00001598 00000100H .idata$4                DATA
 0002:00001698 0000055eH .idata$6                DATA
 0003:00000000 00000068H .data                   DATA
 0003:00000068 0000040cH .bss                    DATA
 0004:00000000 00000060H .rsrc$01                DATA
 0004:00000060 00000330H .rsrc$02                DATA

  Address         Publics by Value              Rva+Base       Lib:Object

 0000:00000000       ___guard_fids_table        00000000     <absolute>
 0000:00000000       ___hybrid_code_map_count   00000000     <absolute>
 0000:00000000       ___guard_longjmp_table     00000000     <absolute>
 0000:00000000       ___hybrid_code_map         00000000     <absolute>
 0000:00000000       ___guard_fids_count        00000000     <absolute>
 0000:00000000       ___guard_iat_count         00000000     <absolute>
 0000:00000000       ___dynamic_value_reloc_table 00000000     <absolute>
 0000:00000000       ___enclave_config          00000000     <absolute>
 0000:00000000       ___guard_longjmp_count     00000000     <absolute>
 0000:00000000       ___guard_iat_table         00000000     <absolute>
 0000:00000000       ___hybrid_auxiliary_iat    00000000     <absolute>
 0000:00000000       ___volatile_metadata       00000000     <absolute>
 0000:00000001       ___safe_se_handler_count   00000001     <absolute>
 0000:00000100       ___guard_flags             00000100     <absolute>
 0000:00000000       ___ImageBase               10000000     <linker-defined>
 0001:00000000       _Java_com_sun_management_internal_DiagnosticCommandImpl_executeDiagnosticCommand@12 10001000 f   DiagnosticCommandImpl.obj
 0001:00000016       _Java_com_sun_management_internal_DiagnosticCommandImpl_getDiagnosticCommandInfo@12 10001016 f   DiagnosticCommandImpl.obj
 0001:000002d1       _Java_com_sun_management_internal_DiagnosticCommandImpl_getDiagnosticCommands@8 100012d1 f   DiagnosticCommandImpl.obj
 0001:000002e3       _Java_com_sun_management_internal_DiagnosticCommandImpl_setNotificationEnabled@12 100012e3 f   DiagnosticCommandImpl.obj
 0001:0000031a       _getDiagnosticCommandArgumentInfoArray 1000131a f   DiagnosticCommandImpl.obj
 0001:0000053b       _Java_com_sun_management_internal_Flag_getAllFlagNames@8 1000153b f   Flag.obj
 0001:0000054a       _Java_com_sun_management_internal_Flag_getFlags@20 1000154a f   Flag.obj
 0001:00000771       _Java_com_sun_management_internal_Flag_getInternalFlagCount@8 10001771 f   Flag.obj
 0001:00000784       _Java_com_sun_management_internal_Flag_initialize@8 10001784 f   Flag.obj
 0001:00000810       _Java_com_sun_management_internal_Flag_setBooleanValue@16 10001810 f   Flag.obj
 0001:00000833       _Java_com_sun_management_internal_Flag_setDoubleValue@20 10001833 f   Flag.obj
 0001:00000858       _Java_com_sun_management_internal_Flag_setLongValue@20 10001858 f   Flag.obj
 0001:00000873       _Java_com_sun_management_internal_Flag_setStringValue@16 10001873 f   Flag.obj
 0001:000008b8       _Java_com_sun_management_internal_GarbageCollectorExtImpl_setNotificationEnabled@16 100018b8 f   GarbageCollectorExtImpl.obj
 0001:000008f4       _Java_com_sun_management_internal_GcInfoBuilder_fillGcAttributeInfo@28 100018f4 f   GcInfoBuilder.obj
 0001:00000a84       _Java_com_sun_management_internal_GcInfoBuilder_getLastGcInfo0@32 10001a84 f   GcInfoBuilder.obj
 0001:00000d1b       _Java_com_sun_management_internal_GcInfoBuilder_getNumGcExtAttributes@12 10001d1b f   GcInfoBuilder.obj
 0001:00000d4c       _Java_com_sun_management_internal_HotSpotDiagnostic_dumpHeap0@16 10001d4c f   HotSpotDiagnostic.obj
 0001:00000d83       _Java_com_sun_management_internal_OperatingSystemImpl_getCommittedVirtualMemorySize0@8 10001d83 f   OperatingSystemImpl.obj
 0001:00000dc2       _Java_com_sun_management_internal_OperatingSystemImpl_getFreePhysicalMemorySize0@8 10001dc2 f   OperatingSystemImpl.obj
 0001:00000df7       _Java_com_sun_management_internal_OperatingSystemImpl_getFreeSwapSpaceSize0@8 10001df7 f   OperatingSystemImpl.obj
 0001:00000e2c       _Java_com_sun_management_internal_OperatingSystemImpl_getProcessCpuLoad0@8 10001e2c f   OperatingSystemImpl.obj
 0001:00000e99       _Java_com_sun_management_internal_OperatingSystemImpl_getProcessCpuTime0@8 10001e99 f   OperatingSystemImpl.obj
 0001:00000ee6       _Java_com_sun_management_internal_OperatingSystemImpl_getSystemCpuLoad0@8 10001ee6 f   OperatingSystemImpl.obj
 0001:00000f40       _Java_com_sun_management_internal_OperatingSystemImpl_getTotalPhysicalMemorySize0@8 10001f40 f   OperatingSystemImpl.obj
 0001:00000f75       _Java_com_sun_management_internal_OperatingSystemImpl_getTotalSwapSpaceSize0@8 10001f75 f   OperatingSystemImpl.obj
 0001:00000faa       _Java_com_sun_management_internal_OperatingSystemImpl_initialize0@8 10001faa f   OperatingSystemImpl.obj
 0001:00000fd1       ___local_stdio_printf_options 10001fd1 f i OperatingSystemImpl.obj
 0001:00000fd7       __snprintf                 10001fd7 f i OperatingSystemImpl.obj
 0001:00000ff1       __vsnprintf                10001ff1 f i OperatingSystemImpl.obj
 0001:0000100c       __vsnprintf_l              1000200c f i OperatingSystemImpl.obj
 0001:00001a7f       _JNI_OnLoad@8              10002a7f f   management_ext.obj
 0001:00001add       _JVM_GetManagement@4       10002add f   jvm:jvm.dll
 0001:00001ae3       _GetProcessMemoryInfo@12   10002ae3 f   psapi:PSAPI.DLL
 0001:00001ae9       _JNU_ThrowByName@12        10002ae9 f   java:java.dll
 0001:00001aef       _JNU_ThrowNullPointerException@8 10002aef f   java:java.dll
 0001:00001af5       _JNU_ThrowOutOfMemoryError@8 10002af5 f   java:java.dll
 0001:00001afb       _JNU_NewObjectByName       10002afb f   java:java.dll
 0001:00001b01       _JNU_ThrowIllegalArgumentException@8 10002b01 f   java:java.dll
 0001:00001b07       _JNU_ThrowInternalError@8  10002b07 f   java:java.dll
 0001:00001b0d       _JNU_GetStaticFieldByName@20 10002b0d f   java:java.dll
 0001:00001b13       @__security_check_cookie@4 10002b13 f   MSVCRT:secchk.obj
 0001:00001b30       __allmul                   10002b30 f   MSVCRT:llmul.obj
 0001:00001e84       __DllMainCRTStartup@12     10002e84 f   MSVCRT:dll_dllmain.obj
 0001:00001ea7       ___raise_securityfailure   10002ea7 f   MSVCRT:gs_report.obj
 0001:00001ecf       ___report_gsfailure        10002ecf f   MSVCRT:gs_report.obj
 0001:00002015       ___security_init_cookie    10003015 f   MSVCRT:gs_support.obj
 0001:00002060       _DllMain@12                10003060 f   MSVCRT:dll_dllmain_stub.obj
 0001:00002082       ?__scrt_initialize_type_info@@YAXXZ 10003082 f   MSVCRT:tncleanup.obj
 0001:0000208e       ?__scrt_uninitialize_type_info@@YAXXZ 1000308e f   MSVCRT:tncleanup.obj
 0001:0000209a       ___local_stdio_scanf_options 1000309a f i MSVCRT:default_local_stdio_options.obj
 0001:000020a0       ___scrt_initialize_default_local_stdio_options 100030a0 f   MSVCRT:default_local_stdio_options.obj
 0001:00002101       ___scrt_acquire_startup_lock 10003101 f   MSVCRT:utility.obj
 0001:00002133       ___scrt_dllmain_after_initialize_c 10003133 f   MSVCRT:utility.obj
 0001:0000215e       ___scrt_dllmain_before_initialize_c 1000315e f   MSVCRT:utility.obj
 0001:0000216c       ___scrt_dllmain_crt_thread_attach 1000316c f   MSVCRT:utility.obj
 0001:0000218b       ___scrt_dllmain_crt_thread_detach 1000318b f   MSVCRT:utility.obj
 0001:00002198       ___scrt_dllmain_exception_filter 10003198 f   MSVCRT:utility.obj
 0001:000021cc       ___scrt_dllmain_uninitialize_c 100031cc f   MSVCRT:utility.obj
 0001:000021ef       ___scrt_dllmain_uninitialize_critical 100031ef f   MSVCRT:utility.obj
 0001:000021fc       ___scrt_initialize_crt     100031fc f   MSVCRT:utility.obj
 0001:00002235       ___scrt_initialize_onexit_tables 10003235 f   MSVCRT:utility.obj
 0001:000022da       ___scrt_is_nonwritable_in_current_image 100032da f   MSVCRT:utility.obj
 0001:0000236e       ___scrt_release_startup_lock 1000336e f   MSVCRT:utility.obj
 0001:0000238b       ___scrt_uninitialize_crt   1000338b f   MSVCRT:utility.obj
 0001:000023b3       ___scrt_get_dyn_tls_init_callback 100033b3 f   MSVCRT:dyn_tls_init.obj
 0001:000023b9       ___scrt_fastfail           100033b9 f   MSVCRT:utility_desktop.obj
 0001:000024d3       __crt_debugger_hook        100034d3 f   MSVCRT:utility_desktop.obj
 0001:000024db       __RTC_Initialize           100034db f   MSVCRT:initsect.obj
 0001:00002507       __RTC_Terminate            10003507 f   MSVCRT:initsect.obj
 0001:00002540       __SEH_prolog4              10003540 f   MSVCRT:sehprolg4.obj
 0001:00002586       __SEH_epilog4              10003586 f   MSVCRT:sehprolg4.obj
 0001:0000259b       __except_handler4          1000359b f   MSVCRT:chandler4gs.obj
 0001:000025be       @_guard_check_icall_nop@4  100035be f i MSVCRT:guard_support.obj
 0001:000025bf       ___isa_available_init      100035bf f   MSVCRT:cpu_disp.obj
 0001:00002756       __get_startup_argv_mode    10003756 f   MSVCRT:argv_mode.obj
 0001:0000275a       ___scrt_is_ucrt_dll_in_use 1000375a f   MSVCRT:ucrt_detection.obj
 0001:00002766       _IsProcessorFeaturePresent@4 10003766 f   kernel32:KERNEL32.dll
 0001:0000276c       _memset                    1000376c f   vcruntime:VCRUNTIME140.dll
 0001:00002772       _strrchr                   10003772 f   vcruntime:VCRUNTIME140.dll
 0001:00002778       ___std_type_info_destroy_list 10003778 f   vcruntime:VCRUNTIME140.dll
 0001:0000277e       __except_handler4_common   1000377e f   vcruntime:VCRUNTIME140.dll
 0001:00002784       _strlen                    10003784 f   ucrt:api-ms-win-crt-string-l1-1-0.dll
 0001:0000278a       __initterm                 1000378a f   ucrt:api-ms-win-crt-runtime-l1-1-0.dll
 0001:00002790       __initterm_e               10003790 f   ucrt:api-ms-win-crt-runtime-l1-1-0.dll
 0001:00002796       __seh_filter_dll           10003796 f   ucrt:api-ms-win-crt-runtime-l1-1-0.dll
 0001:0000279c       __configure_narrow_argv    1000379c f   ucrt:api-ms-win-crt-runtime-l1-1-0.dll
 0001:000027a2       __initialize_narrow_environment 100037a2 f   ucrt:api-ms-win-crt-runtime-l1-1-0.dll
 0001:000027a8       __initialize_onexit_table  100037a8 f   ucrt:api-ms-win-crt-runtime-l1-1-0.dll
 0001:000027ae       __execute_onexit_table     100037ae f   ucrt:api-ms-win-crt-runtime-l1-1-0.dll
 0001:000027b4       __cexit                    100037b4 f   ucrt:api-ms-win-crt-runtime-l1-1-0.dll
 0001:000027ba       ___acrt_initialize         100037ba f   MSVCRT:ucrt_stubs.obj
 0001:000027ba       ___acrt_uninitialize_critical 100037ba f   MSVCRT:ucrt_stubs.obj
 0001:000027ba       ___scrt_stub_for_acrt_thread_attach 100037ba f   MSVCRT:ucrt_stubs.obj
 0001:000027ba       ___vcrt_thread_attach      100037ba f   MSVCRT:ucrt_stubs.obj
 0001:000027ba       ___scrt_stub_for_acrt_thread_detach 100037ba f   MSVCRT:ucrt_stubs.obj
 0001:000027ba       ___scrt_stub_for_acrt_uninitialize_critical 100037ba f   MSVCRT:ucrt_stubs.obj
 0001:000027ba       ___acrt_thread_attach      100037ba f   MSVCRT:ucrt_stubs.obj
 0001:000027ba       ___acrt_thread_detach      100037ba f   MSVCRT:ucrt_stubs.obj
 0001:000027ba       ___vcrt_thread_detach      100037ba f   MSVCRT:ucrt_stubs.obj
 0001:000027ba       ___vcrt_uninitialize       100037ba f   MSVCRT:ucrt_stubs.obj
 0001:000027ba       ___acrt_uninitialize       100037ba f   MSVCRT:ucrt_stubs.obj
 0001:000027ba       ___scrt_stub_for_acrt_uninitialize 100037ba f   MSVCRT:ucrt_stubs.obj
 0001:000027ba       ___vcrt_uninitialize_critical 100037ba f   MSVCRT:ucrt_stubs.obj
 0001:000027ba       ___scrt_stub_for_acrt_initialize 100037ba f   MSVCRT:ucrt_stubs.obj
 0001:000027ba       ___vcrt_initialize         100037ba f   MSVCRT:ucrt_stubs.obj
 0001:000027bd       __is_c_termination_complete 100037bd f   MSVCRT:ucrt_stubs.obj
 0001:000027bd       ___scrt_stub_for_is_c_termination_complete 100037bd f   MSVCRT:ucrt_stubs.obj
 0002:00000000       __imp__InitializeSListHead@4 10004000     kernel32:KERNEL32.dll
 0002:00000004       __imp__DisableThreadLibraryCalls@4 10004004     kernel32:KERNEL32.dll
 0002:00000008       __imp__GetSystemTimeAsFileTime@4 10004008     kernel32:KERNEL32.dll
 0002:0000000c       __imp__GetCurrentProcessId@0 1000400c     kernel32:KERNEL32.dll
 0002:00000010       __imp__QueryPerformanceCounter@4 10004010     kernel32:KERNEL32.dll
 0002:00000014       __imp__IsProcessorFeaturePresent@4 10004014     kernel32:KERNEL32.dll
 0002:00000018       __imp__TerminateProcess@8  10004018     kernel32:KERNEL32.dll
 0002:0000001c       __imp__SetUnhandledExceptionFilter@4 1000401c     kernel32:KERNEL32.dll
 0002:00000020       __imp__UnhandledExceptionFilter@4 10004020     kernel32:KERNEL32.dll
 0002:00000024       __imp__LoadLibraryA@4      10004024     kernel32:KERNEL32.dll
 0002:00000028       __imp__GetLastError@0      10004028     kernel32:KERNEL32.dll
 0002:0000002c       __imp__InitializeCriticalSection@4 1000402c     kernel32:KERNEL32.dll
 0002:00000030       __imp__EnterCriticalSection@4 10004030     kernel32:KERNEL32.dll
 0002:00000034       __imp__LeaveCriticalSection@4 10004034     kernel32:KERNEL32.dll
 0002:00000038       __imp__GetProcessTimes@20  10004038     kernel32:KERNEL32.dll
 0002:0000003c       __imp__GetCurrentProcess@0 1000403c     kernel32:KERNEL32.dll
 0002:00000040       __imp__GetCurrentThreadId@0 10004040     kernel32:KERNEL32.dll
 0002:00000044       __imp__GlobalMemoryStatusEx@4 10004044     kernel32:KERNEL32.dll
 0002:00000048       __imp__GetSystemInfo@4     10004048     kernel32:KERNEL32.dll
 0002:0000004c       __imp__FreeLibrary@4       1000404c     kernel32:KERNEL32.dll
 0002:00000050       __imp__GetModuleFileNameA@12 10004050     kernel32:KERNEL32.dll
 0002:00000054       __imp__GetProcAddress@8    10004054     kernel32:KERNEL32.dll
 0002:00000058       __imp__IsDebuggerPresent@0 10004058     kernel32:KERNEL32.dll
 0002:0000005c       \177KERNEL32_NULL_THUNK_DATA 1000405c     kernel32:KERNEL32.dll
 0002:00000060       __imp__GetProcessMemoryInfo@12 10004060     psapi:PSAPI.DLL
 0002:00000064       \177PSAPI_NULL_THUNK_DATA  10004064     psapi:PSAPI.DLL
 0002:00000068       __imp___except_handler4_common 10004068     vcruntime:VCRUNTIME140.dll
 0002:0000006c       __imp____std_type_info_destroy_list 1000406c     vcruntime:VCRUNTIME140.dll
 0002:00000070       __imp__strrchr             10004070     vcruntime:VCRUNTIME140.dll
 0002:00000074       __imp__memset              10004074     vcruntime:VCRUNTIME140.dll
 0002:00000078       \177VCRUNTIME140_NULL_THUNK_DATA 10004078     vcruntime:VCRUNTIME140.dll
 0002:0000007c       __imp__itoa                1000407c     ucrt:api-ms-win-crt-convert-l1-1-0.dll
 0002:0000007c       __imp___itoa               1000407c     ucrt:api-ms-win-crt-convert-l1-1-0.dll
 0002:00000080       \177api-ms-win-crt-convert-l1-1-0_NULL_THUNK_DATA 10004080     ucrt:api-ms-win-crt-convert-l1-1-0.dll
 0002:00000084       __imp__calloc              10004084     ucrt:api-ms-win-crt-heap-l1-1-0.dll
 0002:00000088       __imp__free                10004088     ucrt:api-ms-win-crt-heap-l1-1-0.dll
 0002:0000008c       __imp__malloc              1000408c     ucrt:api-ms-win-crt-heap-l1-1-0.dll
 0002:00000090       \177api-ms-win-crt-heap-l1-1-0_NULL_THUNK_DATA 10004090     ucrt:api-ms-win-crt-heap-l1-1-0.dll
 0002:00000094       __imp___execute_onexit_table 10004094     ucrt:api-ms-win-crt-runtime-l1-1-0.dll
 0002:00000098       __imp___cexit              10004098     ucrt:api-ms-win-crt-runtime-l1-1-0.dll
 0002:0000009c       __imp___initialize_onexit_table 1000409c     ucrt:api-ms-win-crt-runtime-l1-1-0.dll
 0002:000000a0       __imp___initialize_narrow_environment 100040a0     ucrt:api-ms-win-crt-runtime-l1-1-0.dll
 0002:000000a4       __imp___configure_narrow_argv 100040a4     ucrt:api-ms-win-crt-runtime-l1-1-0.dll
 0002:000000a8       __imp___initterm_e         100040a8     ucrt:api-ms-win-crt-runtime-l1-1-0.dll
 0002:000000ac       __imp___seh_filter_dll     100040ac     ucrt:api-ms-win-crt-runtime-l1-1-0.dll
 0002:000000b0       __imp___getpid             100040b0     ucrt:api-ms-win-crt-runtime-l1-1-0.dll
 0002:000000b4       __imp___initterm           100040b4     ucrt:api-ms-win-crt-runtime-l1-1-0.dll
 0002:000000b8       \177api-ms-win-crt-runtime-l1-1-0_NULL_THUNK_DATA 100040b8     ucrt:api-ms-win-crt-runtime-l1-1-0.dll
 0002:000000bc       __imp____stdio_common_vsprintf 100040bc     ucrt:api-ms-win-crt-stdio-l1-1-0.dll
 0002:000000c0       \177api-ms-win-crt-stdio-l1-1-0_NULL_THUNK_DATA 100040c0     ucrt:api-ms-win-crt-stdio-l1-1-0.dll
 0002:000000c4       __imp__strlen              100040c4     ucrt:api-ms-win-crt-string-l1-1-0.dll
 0002:000000c8       __imp__strncpy             100040c8     ucrt:api-ms-win-crt-string-l1-1-0.dll
 0002:000000cc       \177api-ms-win-crt-string-l1-1-0_NULL_THUNK_DATA 100040cc     ucrt:api-ms-win-crt-string-l1-1-0.dll
 0002:000000d0       __imp__clock               100040d0     ucrt:api-ms-win-crt-time-l1-1-0.dll
 0002:000000d4       \177api-ms-win-crt-time-l1-1-0_NULL_THUNK_DATA 100040d4     ucrt:api-ms-win-crt-time-l1-1-0.dll
 0002:000000d8       __imp__JNU_ThrowIllegalArgumentException@8 100040d8     java:java.dll
 0002:000000dc       __imp__JNU_ThrowInternalError@8 100040dc     java:java.dll
 0002:000000e0       __imp__JNU_ThrowNullPointerException@8 100040e0     java:java.dll
 0002:000000e4       __imp__JNU_GetStaticFieldByName@20 100040e4     java:java.dll
 0002:000000e8       __imp__JNU_ThrowByName@12  100040e8     java:java.dll
 0002:000000ec       __imp__JNU_ThrowOutOfMemoryError@8 100040ec     java:java.dll
 0002:000000f0       __imp__JNU_NewObjectByName 100040f0     java:java.dll
 0002:000000f4       \177java_NULL_THUNK_DATA   100040f4     java:java.dll
 0002:000000f8       __imp__JVM_GetManagement@4 100040f8     jvm:jvm.dll
 0002:000000fc       \177jvm_NULL_THUNK_DATA    100040fc     jvm:jvm.dll
 0002:00000100       ___guard_check_icall_fptr  10004100     MSVCRT:guard_support.obj
 0002:00000104       ___xc_a                    10004104     MSVCRT:initializers.obj
 0002:00000108       ___xc_z                    10004108     MSVCRT:initializers.obj
 0002:0000010c       ___xi_a                    1000410c     MSVCRT:initializers.obj
 0002:00000110       ___xi_z                    10004110     MSVCRT:initializers.obj
 0002:00000114       ___xp_a                    10004114     MSVCRT:initializers.obj
 0002:00000118       ___xp_z                    10004118     MSVCRT:initializers.obj
 0002:0000011c       ___xt_a                    1000411c     MSVCRT:initializers.obj
 0002:00000120       ___xt_z                    10004120     MSVCRT:initializers.obj
 0002:00000130       ??_C@_0FA@KDGODBFA@JMX?5interface?5to?5diagnostic?5fra@ 10004130     DiagnosticCommandImpl.obj
 0002:00000180       ??_C@_0CI@LDDEGNGM@java?1lang?1UnsupportedOperationE@ 10004180     DiagnosticCommandImpl.obj
 0002:000001a8       ??_C@_0DK@NFGDGGMJ@com?1sun?1management?1internal?1Dia@ 100041a8     DiagnosticCommandImpl.obj
 0002:000001e8       ??_C@_0FA@HCGGLJHE@?$CILjava?1lang?1String?$DLLjava?1lang?1S@ 100041e8     DiagnosticCommandImpl.obj
 0002:00000238       ??_C@_0BB@PPEHBGID@java?1util?1Arrays@ 10004238     DiagnosticCommandImpl.obj
 0002:0000024c       ??_C@_0CG@HHOJOFBP@?$CI?$FLLjava?1lang?1Object?$DL?$CJLjava?1util@ 1000424c     DiagnosticCommandImpl.obj
 0002:00000274       ??_C@_06ECNHPIF@asList@    10004274     DiagnosticCommandImpl.obj
 0002:0000027c       ??_C@_0BF@IEOOPILA@Invalid?5String?5Array@ 1000427c     DiagnosticCommandImpl.obj
 0002:00000294       ??_C@_0DC@EEHIJFOL@com?1sun?1management?1internal?1Dia@ 10004294     DiagnosticCommandImpl.obj
 0002:000002c8       ??_C@_0IB@BKJILNLP@?$CILjava?1lang?1String?$DLLjava?1lang?1S@ 100042c8     DiagnosticCommandImpl.obj
 0002:0000034c       ??_C@_0CF@MADHDJEK@Lcom?1sun?1management?1VMOption$Or@ 1000434c     Flag.obj
 0002:00000374       ??_C@_0CD@CEAHIHPC@com?1sun?1management?1VMOption$Ori@ 10004374     Flag.obj
 0002:00000398       ??_C@_07MGCPDNLD@DEFAULT@  10004398     Flag.obj
 0002:000003a0       ??_C@_0M@BODHNBPF@VM_CREATION@ 100043a0     Flag.obj
 0002:000003ac       ??_C@_0L@HNPILAMG@MANAGEMENT@ 100043ac     Flag.obj
 0002:000003b8       ??_C@_0M@FDANMCLI@ENVIRON_VAR@ 100043b8     Flag.obj
 0002:000003c4       ??_C@_0M@CEBLKBIO@CONFIG_FILE@ 100043c4     Flag.obj
 0002:000003d0       ??_C@_09ILMJHCBE@ERGONOMIC@ 100043d0     Flag.obj
 0002:000003dc       ??_C@_0BB@ICEJIAEF@ATTACH_ON_DEMAND@ 100043dc     Flag.obj
 0002:000003f0       ??_C@_05NNNMIPMB@OTHER@    100043f0     Flag.obj
 0002:000003f8       ??_C@_0CB@NMENEKD@com?1sun?1management?1internal?1Fla@ 100043f8     Flag.obj
 0002:00000420       ??_C@_0EO@OCMOFBBM@?$CILjava?1lang?1String?$DLLjava?1lang?1O@ 10004420     Flag.obj
 0002:00000470       ??_C@_04LHKBAEFM@?$CIZ?$CJV@ 10004470     Flag.obj
 0002:00000478       ??_C@_0BC@DDPBLLCP@java?1lang?1Boolean@ 10004478     Flag.obj
 0002:0000048c       ??_C@_04OHLIFDMD@?$CIJ?$CJV@ 1000448c     Flag.obj
 0002:00000494       ??_C@_0P@MLLHBNNC@java?1lang?1Long@ 10004494     Flag.obj
 0002:000004a4       ??_C@_04HGHCEPA@?$CID?$CJV@ 100044a4     Flag.obj
 0002:000004ac       ??_C@_0BB@JKEOLFJD@java?1lang?1Double@ 100044ac     Flag.obj
 0002:000004c0       ??_C@_0CJ@FEKHENIJ@Number?5of?5Flag?5objects?5created?5@ 100044c0     Flag.obj
 0002:000004ec       ??_C@_0BO@EOMDLAMD@Invalid?5GarbageCollectorMBean@ 100044ec     GarbageCollectorExtImpl.obj
 0002:0000050c       ??_C@_0P@CCHCOPNE@java?1lang?1Byte@ 1000450c     GcInfoBuilder.obj
 0002:0000051c       ??_C@_04CCAMHLCM@?$CIB?$CJV@ 1000451c     GcInfoBuilder.obj
 0002:00000524       ??_C@_0BC@OHJKABOO@java?1lang?1Integer@ 10004524     GcInfoBuilder.obj
 0002:00000538       ??_C@_04PFANPMCN@?$CII?$CJV@ 10004538     GcInfoBuilder.obj
 0002:00000540       ??_C@_0BA@MBLENCLH@java?1lang?1Short@ 10004540     GcInfoBuilder.obj
 0002:00000550       ??_C@_04MKKJELNG@?$CIS?$CJV@ 10004550     GcInfoBuilder.obj
 0002:00000558       ??_C@_0BA@HJEPPKHG@java?1lang?1Float@ 10004558     GcInfoBuilder.obj
 0002:00000568       ??_C@_0BE@GKIHCGPM@java?1lang?1Character@ 10004568     GcInfoBuilder.obj
 0002:0000057c       ??_C@_04JKLABMEJ@?$CIC?$CJV@ 1000457c     GcInfoBuilder.obj
 0002:00000584       ??_C@_0BH@KCPAAINP@Invalid?5num_attributes@ 10004584     GcInfoBuilder.obj
 0002:0000059c       ??_C@_0BK@KGMIKEPP@Unexpected?5num_attributes@ 1000459c     GcInfoBuilder.obj
 0002:000005b8       ??_C@_0BG@HCNJLLGG@Invalid?5ext_att_count@ 100045b8     GcInfoBuilder.obj
 0002:000005d0       ??_C@_0BL@CHBGEDL@Unsupported?5attribute?5type@ 100045d0     GcInfoBuilder.obj
 0002:000005f0       ??_C@_0IL@DNFKACMC@?$CILcom?1sun?1management?1internal?1G@ 100045f0     GcInfoBuilder.obj
 0002:0000067c       ??_C@_0BK@LAMMNKDJ@com?1sun?1management?1GcInfo@ 1000467c     GcInfoBuilder.obj
 0002:000006c4       ??_C@_06NELKLDPM@?2?$CFs?2?$CFs@ 100046c4     OperatingSystemImpl.obj
 0002:000006cc       ??_C@_0L@MLLIHFJC@?2?$CFs?$CI?$CFs?$CJ?2?$CFs@ 100046cc     OperatingSystemImpl.obj
 0002:000006d8       ??_C@_0O@JCGOHBMM@?2?$CFs?$CI?$CFs?$CD?$CFs?$CJ?2?$CFs@ 100046d8     OperatingSystemImpl.obj
 0002:000006e8       ??_C@_0P@CIDEDEDD@PdhAddCounterA@ 100046e8     OperatingSystemImpl.obj
 0002:000006f8       ??_C@_0O@HFNMDKII@PdhOpenQueryA@ 100046f8     OperatingSystemImpl.obj
 0002:00000708       ??_C@_0O@EGDBAKJC@PdhCloseQuery@ 10004708     OperatingSystemImpl.obj
 0002:00000718       ??_C@_0BE@GPNBOCHE@PdhCollectQueryData@ 10004718     OperatingSystemImpl.obj
 0002:0000072c       ??_C@_0BM@EOJADGC@PdhGetFormattedCounterValue@ 1000472c     OperatingSystemImpl.obj
 0002:00000748       ??_C@_0BE@BJADGCJL@PdhEnumObjectItemsA@ 10004748     OperatingSystemImpl.obj
 0002:0000075c       ??_C@_0BB@EBECGLNG@PdhRemoveCounter@ 1000475c     OperatingSystemImpl.obj
 0002:00000770       ??_C@_0BK@BKCEHIDJ@PdhLookupPerfNameByIndexA@ 10004770     OperatingSystemImpl.obj
 0002:0000078c       ??_C@_02DPKJAMEF@?$CFd@    1000478c     OperatingSystemImpl.obj
 0002:00000790       ??_C@_07OPODLDBJ@pdh?4dll@ 10004790     OperatingSystemImpl.obj
 0002:00000798       __real@3ff0000000000000    10004798     OperatingSystemImpl.obj
 0002:000007a0       __real@4059000000000000    100047a0     OperatingSystemImpl.obj
 0002:000007a8       __real@bff0000000000000    100047a8     OperatingSystemImpl.obj
 0002:000007b0       __xmm@41f00000000000000000000000000000 100047b0     OperatingSystemImpl.obj
 0002:000007c0       ??_C@_0BP@KJIDAONK@Unsupported?5Management?5version@ 100047c0     management_ext.obj
 0002:000007e0       __pDefaultRawDllMain       100047e0     MSVCRT:dll_dllmain.obj
 0002:000007e0       __pRawDllMain              100047e0     MSVCRT:dll_dllmain.obj
 0002:00000860       __load_config_used         10004860     MSVCRT:loadcfg.obj
 0002:00000900       ___safe_se_handler_table   10004900     <linker-defined>
 0002:00000b90       ___rtc_iaa                 10004b90     MSVCRT:initsect.obj
 0002:00000b94       ___rtc_izz                 10004b94     MSVCRT:initsect.obj
 0002:00000b98       ___rtc_taa                 10004b98     MSVCRT:initsect.obj
 0002:00000b9c       ___rtc_tzz                 10004b9c     MSVCRT:initsect.obj
 0002:000014a8       __IMPORT_DESCRIPTOR_jvm    100054a8     jvm:jvm.dll
 0002:000014bc       __IMPORT_DESCRIPTOR_PSAPI  100054bc     psapi:PSAPI.DLL
 0002:000014d0       __IMPORT_DESCRIPTOR_java   100054d0     java:java.dll
 0002:000014e4       __IMPORT_DESCRIPTOR_KERNEL32 100054e4     kernel32:KERNEL32.dll
 0002:000014f8       __IMPORT_DESCRIPTOR_VCRUNTIME140 100054f8     vcruntime:VCRUNTIME140.dll
 0002:0000150c       __IMPORT_DESCRIPTOR_api-ms-win-crt-heap-l1-1-0 1000550c     ucrt:api-ms-win-crt-heap-l1-1-0.dll
 0002:00001520       __IMPORT_DESCRIPTOR_api-ms-win-crt-stdio-l1-1-0 10005520     ucrt:api-ms-win-crt-stdio-l1-1-0.dll
 0002:00001534       __IMPORT_DESCRIPTOR_api-ms-win-crt-string-l1-1-0 10005534     ucrt:api-ms-win-crt-string-l1-1-0.dll
 0002:00001548       __IMPORT_DESCRIPTOR_api-ms-win-crt-time-l1-1-0 10005548     ucrt:api-ms-win-crt-time-l1-1-0.dll
 0002:0000155c       __IMPORT_DESCRIPTOR_api-ms-win-crt-runtime-l1-1-0 1000555c     ucrt:api-ms-win-crt-runtime-l1-1-0.dll
 0002:00001570       __IMPORT_DESCRIPTOR_api-ms-win-crt-convert-l1-1-0 10005570     ucrt:api-ms-win-crt-convert-l1-1-0.dll
 0002:00001584       __NULL_IMPORT_DESCRIPTOR   10005584     jvm:jvm.dll
 0003:00000040       __fltused                  10006040     MSVCRT:fltused.obj
 0003:00000050       ___security_cookie_complement 10006050     MSVCRT:gs_cookie.obj
 0003:00000054       ___security_cookie         10006054     MSVCRT:gs_cookie.obj
 0003:00000058       ___scrt_native_dllmain_reason 10006058     MSVCRT:utility.obj
 0003:00000060       ___isa_enabled             10006060     MSVCRT:cpu_disp.obj
 0003:00000064       ___scrt_ucrt_dll_is_in_use 10006064     MSVCRT:ucrt_stubs.obj
 0003:000000f8       _jmm_interface             100060f8     management_ext.obj
 0003:000000fc       _jmm_version               100060fc     management_ext.obj
 0003:00000100       _jvm                       10006100     management_ext.obj
 0003:00000428       ?__type_info_root_node@@3U__type_info_node@@A 10006428     MSVCRT:tncleanup.obj
 0003:00000430       ?_OptionsStorage@?1??__local_stdio_scanf_options@@9@4_KA 10006430     MSVCRT:default_local_stdio_options.obj
 0003:00000438       ___scrt_current_native_startup_state 10006438     MSVCRT:utility.obj
 0003:0000043c       ___scrt_native_startup_lock 1000643c     MSVCRT:utility.obj
 0003:0000045c       ___scrt_debugger_hook_flag 1000645c     MSVCRT:utility_desktop.obj
 0003:00000460       ___isa_available           10006460     MSVCRT:cpu_disp.obj
 0003:00000464       ___favor                   10006464     MSVCRT:cpu_disp.obj
 0003:00000468       ?_OptionsStorage@?1??__local_stdio_printf_options@@9@9 10006468     <common>
 0003:00000470       ___dyn_tls_init_callback   10006470     <common>

 entry point at        0001:00001e84

 Static symbols

 0000:ffff7000       .debug$S                   10000000     ucrt:api-ms-win-crt-runtime-l1-1-0.dll
 0000:ffff7000       .debug$S                   10000000     kernel32:KERNEL32.dll
 0000:ffff7000       .debug$S                   10000000     kernel32:KERNEL32.dll
 0000:ffff7000       .debug$S                   10000000     kernel32:KERNEL32.dll
 0000:ffff7000       .debug$S                   10000000     kernel32:KERNEL32.dll
 0000:ffff7000       .debug$S                   10000000     kernel32:KERNEL32.dll
 0000:ffff7000       .debug$S                   10000000     kernel32:KERNEL32.dll
 0000:ffff7000       .debug$S                   10000000     kernel32:KERNEL32.dll
 0000:ffff7000       .debug$S                   10000000     kernel32:KERNEL32.dll
 0000:ffff7000       .debug$S                   10000000     kernel32:KERNEL32.dll
 0000:ffff7000       .debug$S                   10000000     kernel32:KERNEL32.dll
 0000:ffff7000       .debug$S                   10000000     kernel32:KERNEL32.dll
 0000:ffff7000       .debug$S                   10000000     kernel32:KERNEL32.dll
 0000:ffff7000       .debug$S                   10000000     kernel32:KERNEL32.dll
 0000:ffff7000       .debug$S                   10000000     kernel32:KERNEL32.dll
 0000:ffff7000       .debug$S                   10000000     kernel32:KERNEL32.dll
 0000:ffff7000       .debug$S                   10000000     kernel32:KERNEL32.dll
 0000:ffff7000       .debug$S                   10000000     kernel32:KERNEL32.dll
 0000:ffff7000       .debug$S                   10000000     jvm:jvm.dll
 0000:ffff7000       .debug$S                   10000000     psapi:PSAPI.DLL
 0000:ffff7000       .debug$S                   10000000     java:java.dll
 0000:ffff7000       .debug$S                   10000000     java:java.dll
 0000:ffff7000       .debug$S                   10000000     java:java.dll
 0000:ffff7000       .debug$S                   10000000     java:java.dll
 0000:ffff7000       .debug$S                   10000000     java:java.dll
 0000:ffff7000       .debug$S                   10000000     java:java.dll
 0000:ffff7000       .debug$S                   10000000     java:java.dll
 0000:ffff7000       .debug$S                   10000000     kernel32:KERNEL32.dll
 0000:ffff7000       .debug$S                   10000000     kernel32:KERNEL32.dll
 0000:ffff7000       .debug$S                   10000000     vcruntime:VCRUNTIME140.dll
 0000:ffff7000       .debug$S                   10000000     vcruntime:VCRUNTIME140.dll
 0000:ffff7000       .debug$S                   10000000     vcruntime:VCRUNTIME140.dll
 0000:ffff7000       .debug$S                   10000000     management_ext.exp
 0000:ffff7000       .debug$S                   10000000     vcruntime:VCRUNTIME140.dll
 0000:ffff7000       .debug$S                   10000000     kernel32:KERNEL32.dll
 0000:ffff7000       .debug$S                   10000000     ucrt:api-ms-win-crt-heap-l1-1-0.dll
 0000:ffff7000       .debug$S                   10000000     kernel32:KERNEL32.dll
 0000:ffff7000       .debug$S                   10000000     kernel32:KERNEL32.dll
 0000:ffff7000       .debug$S                   10000000     kernel32:KERNEL32.dll
 0000:ffff7000       .debug$S                   10000000     kernel32:KERNEL32.dll
 0000:ffff7000       .debug$S                   10000000     ucrt:api-ms-win-crt-convert-l1-1-0.dll
 0000:ffff7000       .debug$S                   10000000     ucrt:api-ms-win-crt-runtime-l1-1-0.dll
 0000:ffff7000       .debug$S                   10000000     ucrt:api-ms-win-crt-runtime-l1-1-0.dll
 0000:ffff7000       .debug$S                   10000000     kernel32:KERNEL32.dll
 0000:ffff7000       .debug$S                   10000000     ucrt:api-ms-win-crt-runtime-l1-1-0.dll
 0000:ffff7000       .debug$S                   10000000     ucrt:api-ms-win-crt-runtime-l1-1-0.dll
 0000:ffff7000       .debug$S                   10000000     ucrt:api-ms-win-crt-runtime-l1-1-0.dll
 0000:ffff7000       .debug$S                   10000000     ucrt:api-ms-win-crt-runtime-l1-1-0.dll
 0000:ffff7000       .debug$S                   10000000     ucrt:api-ms-win-crt-runtime-l1-1-0.dll
 0000:ffff7000       .debug$S                   10000000     ucrt:api-ms-win-crt-runtime-l1-1-0.dll
 0000:ffff7000       .debug$S                   10000000     ucrt:api-ms-win-crt-runtime-l1-1-0.dll
 0000:ffff7000       .debug$S                   10000000     ucrt:api-ms-win-crt-runtime-l1-1-0.dll
 0000:ffff7000       .debug$S                   10000000     ucrt:api-ms-win-crt-runtime-l1-1-0.dll
 0000:ffff7000       .debug$S                   10000000     ucrt:api-ms-win-crt-runtime-l1-1-0.dll
 0000:ffff7000       .debug$S                   10000000     ucrt:api-ms-win-crt-runtime-l1-1-0.dll
 0000:ffff7000       .debug$S                   10000000     ucrt:api-ms-win-crt-time-l1-1-0.dll
 0000:ffff7000       .debug$S                   10000000     ucrt:api-ms-win-crt-heap-l1-1-0.dll
 0000:ffff7000       .debug$S                   10000000     ucrt:api-ms-win-crt-string-l1-1-0.dll
 0000:ffff7000       .debug$S                   10000000     ucrt:api-ms-win-crt-string-l1-1-0.dll
 0000:ffff7000       .debug$S                   10000000     ucrt:api-ms-win-crt-stdio-l1-1-0.dll
 0000:ffff7000       .debug$S                   10000000     ucrt:api-ms-win-crt-heap-l1-1-0.dll
 0001:00000890       _find_origin_constant      10001890 f   Flag.obj
 0001:00000d63       _EnterPdhCriticalSection   10001d63 f   OperatingSystemImpl.obj
 0001:0000103f       _addCounter                1000203f f   OperatingSystemImpl.obj
 0001:00001058       _allocateAndInitializePdhConstants 10002058 f   OperatingSystemImpl.obj
 0001:0000113e       _bindPdhFunctionPointers   1000213e f   OperatingSystemImpl.obj
 0001:000011fe       _currentQueryIndexForProcess 100021fe f   OperatingSystemImpl.obj
 0001:000012e9       _deallocateCPUCounters     100022e9 f   OperatingSystemImpl.obj
 0001:000013a1       _getPdhProcessImageName    100023a1 f   OperatingSystemImpl.obj
 0001:00001446       _getPerformanceData        10002446 f   OperatingSystemImpl.obj
 0001:000014ac       _initializeCPUCounters     100024ac f   OperatingSystemImpl.obj
 0001:000015f9       _initializeMultipleCounterForCPUs 100025f9 f   OperatingSystemImpl.obj
 0001:0000179f       _initializePdhCPUCounters  1000279f f   OperatingSystemImpl.obj
 0001:0000183c       _lookupNameByIndex         1000283c f   OperatingSystemImpl.obj
 0001:0000189e       _makeFullCounterPath       1000289e f   OperatingSystemImpl.obj
 0001:0000196a       _openQuery                 1000296a f   OperatingSystemImpl.obj
 0001:0000197d       _pdhCleanup                1000297d f   OperatingSystemImpl.obj
 0001:000019b0       _pdhInit                   100029b0 f   OperatingSystemImpl.obj
 0001:00001a36       _pdhInitErrorHandler       10002a36 f   OperatingSystemImpl.obj
 0001:00001b30       $$000000                   10002b30     MSVCRT:llmul.obj
 0001:00001b64       ?dllmain_crt_dispatch@@YGHQAUHINSTANCE__@@KQAX@Z 10002b64 f   MSVCRT:dll_dllmain.obj
 0001:00001bb7       ?dllmain_crt_process_attach@@YAHQAUHINSTANCE__@@QAX@Z 10002bb7 f   MSVCRT:dll_dllmain.obj
 0001:00001cc1       ?dllmain_crt_process_detach@@YAH_N@Z 10002cc1 f   MSVCRT:dll_dllmain.obj
 0001:00001d53       ?dllmain_dispatch@@YAHQAUHINSTANCE__@@KQAX@Z 10002d53 f   MSVCRT:dll_dllmain.obj
 0001:00001e59       ?dllmain_raw@@YGHQAUHINSTANCE__@@KQAX@Z 10002e59 f   MSVCRT:dll_dllmain.obj
 0001:00001fc8       ___get_entropy             10002fc8 f   MSVCRT:gs_support.obj
 0001:000020bd       ?find_pe_section@@YAPAU_IMAGE_SECTION_HEADER@@QAEI@Z 100030bd f   MSVCRT:utility.obj
 0001:00002540       $$000000                   10003540     MSVCRT:sehprolg4.obj
 0002:00000698       _MIN_UPDATE_INTERVAL       10004698     OperatingSystemImpl.obj
 0002:0000069c       _PDH_PROCESSOR_IDX         1000469c     OperatingSystemImpl.obj
 0002:000006a0       _PDH_PROCESSOR_TIME_IDX    100046a0     OperatingSystemImpl.obj
 0002:000006a4       _PDH_PROCESS_IDX           100046a4     OperatingSystemImpl.obj
 0002:000006a8       _PDH_ID_PROCESS_IDX        100046a8     OperatingSystemImpl.obj
 0002:000006ac       _OBJECT_COUNTER_FMT        100046ac     OperatingSystemImpl.obj
 0002:000006b0       _OBJECT_COUNTER_FMT_LEN    100046b0     OperatingSystemImpl.obj
 0002:000006b4       _OBJECT_WITH_INSTANCES_COUNTER_FMT 100046b4     OperatingSystemImpl.obj
 0002:000006b8       _OBJECT_WITH_INSTANCES_COUNTER_FMT_LEN 100046b8     OperatingSystemImpl.obj
 0002:000006bc       _PROCESS_OBJECT_INSTANCE_COUNTER_FMT 100046bc     OperatingSystemImpl.obj
 0002:000006c0       _PROCESS_OBJECT_INSTANCE_COUNTER_FMT_LEN 100046c0     OperatingSystemImpl.obj
 0002:000007e4       _GS_ExceptionPointers      100047e4     MSVCRT:gs_report.obj
 0002:00000ba0       __sehtable$?dllmain_crt_process_attach@@YAHQAUHINSTANCE__@@QAX@Z 10004ba0     MSVCRT:dll_dllmain.obj
 0002:00000bc0       __sehtable$?dllmain_crt_process_detach@@YAH_N@Z 10004bc0     MSVCRT:dll_dllmain.obj
 0002:00000be0       __sehtable$?dllmain_dispatch@@YAHQAUHINSTANCE__@@KQAX@Z 10004be0     MSVCRT:dll_dllmain.obj
 0002:00000c00       __sehtable$___scrt_is_nonwritable_in_current_image 10004c00     MSVCRT:utility.obj
 0002:00000c20       .edata                     10004c20     management_ext.exp
 0002:00000c48       rgpv                       10004c48     management_ext.exp
 0002:00000cb4       rgszName                   10004cb4     management_ext.exp
 0002:00000d20       rgwOrd                     10004d20     management_ext.exp
 0002:00000d56       szName                     10004d56     management_ext.exp
 0002:00000d69       $N00001                    10004d69     management_ext.exp
 0002:00000d77       $N00002                    10004d77     management_ext.exp
 0002:00000dcb       $N00003                    10004dcb     management_ext.exp
 0002:00000e1f       $N00004                    10004e1f     management_ext.exp
 0002:00000e6f       $N00005                    10004e6f     management_ext.exp
 0002:00000ec1       $N00006                    10004ec1     management_ext.exp
 0002:00000efa       $N00007                    10004efa     management_ext.exp
 0002:00000f2d       $N00008                    10004f2d     management_ext.exp
 0002:00000f6b       $N00009                    10004f6b     management_ext.exp
 0002:00000f9f       $N00010                    10004f9f     management_ext.exp
 0002:00000fd9       $N00011                    10004fd9     management_ext.exp
 0002:00001012       $N00012                    10005012     management_ext.exp
 0002:00001049       $N00013                    10005049     management_ext.exp
 0002:00001082       $N00014                    10005082     management_ext.exp
 0002:000010d6       $N00015                    100050d6     management_ext.exp
 0002:0000111d       $N00016                    1000511d     management_ext.exp
 0002:0000115f       $N00017                    1000515f     management_ext.exp
 0002:000011a8       $N00018                    100051a8     management_ext.exp
 0002:000011e9       $N00019                    100051e9     management_ext.exp
 0002:00001240       $N00020                    10005240     management_ext.exp
 0002:00001293       $N00021                    10005293     management_ext.exp
 0002:000012e1       $N00022                    100052e1     management_ext.exp
 0002:0000132c       $N00023                    1000532c     management_ext.exp
 0002:00001377       $N00024                    10005377     management_ext.exp
 0002:000013c1       $N00025                    100053c1     management_ext.exp
 0002:00001415       $N00026                    10005415     management_ext.exp
 0002:00001464       $N00027                    10005464     management_ext.exp
 0002:000016b0       .idata$6                   100056b0     jvm:jvm.dll
 0002:000016d0       .idata$6                   100056d0     psapi:PSAPI.DLL
 0002:000017ae       .idata$6                   100057ae     java:java.dll
 0002:000019b8       .idata$6                   100059b8     kernel32:KERNEL32.dll
 0002:00001a14       .idata$6                   10005a14     vcruntime:VCRUNTIME140.dll
 0002:00001b30       .idata$6                   10005b30     ucrt:api-ms-win-crt-heap-l1-1-0.dll
 0002:00001b50       .idata$6                   10005b50     ucrt:api-ms-win-crt-stdio-l1-1-0.dll
 0002:00001b70       .idata$6                   10005b70     ucrt:api-ms-win-crt-string-l1-1-0.dll
 0002:00001b92       .idata$6                   10005b92     ucrt:api-ms-win-crt-time-l1-1-0.dll
 0002:00001bb2       .idata$6                   10005bb2     ucrt:api-ms-win-crt-runtime-l1-1-0.dll
 0002:00001bd4       .idata$6                   10005bd4     ucrt:api-ms-win-crt-convert-l1-1-0.dll
 0003:00000000       ?class_name@?1??setLongValueAtObjectArray@@9@9 10006000     GcInfoBuilder.obj
 0003:00000004       ?signature@?1??setLongValueAtObjectArray@@9@9 10006004     GcInfoBuilder.obj
 0003:00000008       ?class_name@?1??setBooleanValueAtObjectArray@@9@9 10006008     GcInfoBuilder.obj
 0003:0000000c       ?signature@?1??setBooleanValueAtObjectArray@@9@9 1000600c     GcInfoBuilder.obj
 0003:00000010       ?class_name@?1??setByteValueAtObjectArray@@9@9 10006010     GcInfoBuilder.obj
 0003:00000014       ?signature@?1??setByteValueAtObjectArray@@9@9 10006014     GcInfoBuilder.obj
 0003:00000018       ?class_name@?1??setIntValueAtObjectArray@@9@9 10006018     GcInfoBuilder.obj
 0003:0000001c       ?signature@?1??setIntValueAtObjectArray@@9@9 1000601c     GcInfoBuilder.obj
 0003:00000020       ?class_name@?1??setShortValueAtObjectArray@@9@9 10006020     GcInfoBuilder.obj
 0003:00000024       ?signature@?1??setShortValueAtObjectArray@@9@9 10006024     GcInfoBuilder.obj
 0003:00000028       ?class_name@?1??setDoubleValueAtObjectArray@@9@9 10006028     GcInfoBuilder.obj
 0003:0000002c       ?signature@?1??setDoubleValueAtObjectArray@@9@9 1000602c     GcInfoBuilder.obj
 0003:00000030       ?class_name@?1??setFloatValueAtObjectArray@@9@9 10006030     GcInfoBuilder.obj
 0003:00000034       ?signature@?1??setFloatValueAtObjectArray@@9@9 10006034     GcInfoBuilder.obj
 0003:00000038       ?class_name@?1??setCharValueAtObjectArray@@9@9 10006038     GcInfoBuilder.obj
 0003:0000003c       ?signature@?1??setCharValueAtObjectArray@@9@9 1000603c     GcInfoBuilder.obj
 0003:00000068       _default_origin            10006068     Flag.obj
 0003:0000006c       _vm_creation_origin        1000606c     Flag.obj
 0003:00000070       _mgmt_origin               10006070     Flag.obj
 0003:00000074       _envvar_origin             10006074     Flag.obj
 0003:00000078       _config_file_origin        10006078     Flag.obj
 0003:0000007c       _ergo_origin               1000607c     Flag.obj
 0003:00000080       _attach_origin             10006080     Flag.obj
 0003:00000084       _other_origin              10006084     Flag.obj
 0003:00000088       _main_process              10006088     OperatingSystemImpl.obj
 0003:0000008c       _PdhAddCounter_i           1000608c     OperatingSystemImpl.obj
 0003:00000090       _PdhOpenQuery_i            10006090     OperatingSystemImpl.obj
 0003:00000094       _PdhCloseQuery_i           10006094     OperatingSystemImpl.obj
 0003:00000098       _PdhCollectQueryData_i     10006098     OperatingSystemImpl.obj
 0003:0000009c       _PdhGetFormattedCounterValue_i 1000609c     OperatingSystemImpl.obj
 0003:000000a0       _PdhEnumObjectItems_i      100060a0     OperatingSystemImpl.obj
 0003:000000a4       _PdhRemoveCounter_i        100060a4     OperatingSystemImpl.obj
 0003:000000a8       _PdhLookupPerfNameByIndex_i 100060a8     OperatingSystemImpl.obj
 0003:000000ac       _initializationLock        100060ac     OperatingSystemImpl.obj
 0003:000000cc       _pdhProcessImageName       100060cc     OperatingSystemImpl.obj
 0003:000000d0       _pdhIDProcessCounterFmt    100060d0     OperatingSystemImpl.obj
 0003:000000d4       _numberOfJavaProcessesAtInitialization 100060d4     OperatingSystemImpl.obj
 0003:000000d8       _processTotalCPULoad       100060d8     OperatingSystemImpl.obj
 0003:000000dc       _multiCounterCPULoad       100060dc     OperatingSystemImpl.obj
 0003:000000e0       _cpuFactor                 100060e0     OperatingSystemImpl.obj
 0003:000000e8       _numCpus                   100060e8     OperatingSystemImpl.obj
 0003:000000ec       ?myPid@?1??getProcessID@@9@9 100060ec     OperatingSystemImpl.obj
 0003:000000f0       ?initialized@?1??pdhInit@@9@9 100060f0     OperatingSystemImpl.obj
 0003:000000f4       ?initialized@?1??initializePdhCPUCounters@@9@9 100060f4     OperatingSystemImpl.obj
 0003:00000104       ?__proc_attached@@3HA      10006104     MSVCRT:dll_dllmain.obj
 0003:00000108       _GS_ExceptionRecord        10006108     MSVCRT:gs_report.obj
 0003:00000158       _GS_ContextRecord          10006158     MSVCRT:gs_report.obj
 0003:00000440       ?is_initialized_as_dll@@3_NA 10006440     MSVCRT:utility.obj
 0003:00000441       ?module_local_atexit_table_initialized@@3_NA 10006441     MSVCRT:utility.obj
 0003:00000444       ?module_local_atexit_table@@3U_onexit_table_t@@A 10006444     MSVCRT:utility.obj
 0003:00000450       ?module_local_at_quick_exit_table@@3U_onexit_table_t@@A 10006450     MSVCRT:utility.obj
 0004:00000060       $R000000                   10007060     management_ext.dll.res
